:1000000015C0D3C02CC02BC02AC029C029C027C00E
:1000100026C025C024C023C022C021C00001020088
:1000200002000001010000020002010011241FBEB5
:10003000CFEDCDBF10E0A0E6B0E0E6ECFFE003C0FE
:10004000C89531960D92A036B107D1F710E0A0E621
:10005000B0E001C01D92AF38B107E1F74BC1D0CF7E
:100060001F920F920FB60F9211242F933F934F932D
:100070005F936F937F938F939F93AF93BF93EF9310
:10008000FF9380E982BF809185008F5F8093850018
:1000900080918500873010F01092850088B38270BF
:1000A0008C6388BB15BA969828B32270809185001E
:1000B000E82FFF27EF58FF4F808199278F709070AE
:1000C000880F991F880F991F282B28BB80918500C6
:1000D000E82FFF27EF58FF4F808187FD969A809188
:1000E0008500882311F4C09A0EC08091850026E017
:1000F00030E0281B310981E090E002C0880F991F91
:100100002A95E2F785BB80918500833029F469E662
:1001100070E08AE690E01AC080918500843029F46E
:1001200067E870E08EE890E011C08091850085302E
:1001300029F466E870E088E790E008C080918500C7
:10014000863029F46BE770E08BE690E011D0FF91E8
:10015000EF91BF91AF919F918F917F916F915F913F
:100160004F913F912F910F900FBE0F901F901895B8
:10017000B92FA82FF72FE62F8081880F8083859BCA
:1001800003C0808181608083808199278F70907007
:10019000892B11F41C920895808199278F7090709B
:1001A0000F9711F481E08C9308951F920F920FB670
:1001B0000F9211242F933F934F935F936F937F93ED
:1001C0008F939F93AF93BF93EF93FF9315BA18BA92
:1001D00081E082BB11BA90916C00191624F48091D1
:1001E0006D008823E9F080917C0020917D003091A2
:1001F0007E0040917F0050918000823049F420932E
:10020000650030936600409367005093680008C013
:100210002093890030938A0040938B0050938C0088
:1002200019161CF060917C0002C06091700081E0A2
:1002300073D68091890090918A00A0918B00B09133
:100240008C008A2F9B2FAA27BB27682F82E064D6B9
:100250008091890090918A00A0918B00B0918C00D0
:10026000892F9A2FAB2FBB27682F83E055D660913B
:10027000890084E051D68091650090916600A0913C
:100280006700B09168008A2F9B2FAA27BB27682F91
:1002900085E042D68091650090916600A09167004C
:1002A000B0916800892F9A2FAB2FBB27682F86E06B
:1002B00033D66091650087E02FD660916C0088E0AE
:1002C0002BD680E039D6829B03C000008299FDCFF7
:1002D000C7CEFF91EF91BF91AF919F918F917F9189
:1002E0006F915F914F913F912F910F900FBE0F90A3
:1002F0001F901895CFEDD0E0DEBFCDBFF8948CE312
:1003000088BB8FE387BB15BA84BB80E882BB88EDCE
:1003100081BB829B03C000008299FDCF80E090E00A
:100320000000019625E780339207D0F388E181BD74
:100330008FE181BD64EA70E088E033D580E982BF57
:1003400083E083BF89B7826089BF83E285BF8BB7B3
:1003500080648BBF10926A001092690010928E0028
:1003600010928700109278001092860010926B0015
:1003700010927B00109288008FEF80936C00109297
:100380006D00C1E08C2F77D58F3F39F428EE33E034
:1003900040E050E060E08C2F8AD5CF5FC33394F308
:1003A00081E0CAD5682F80937C008F3F29F528EE25
:1003B00033E040E050E02093890030938A0040937E
:1003C0008B0050938C0084E694E1A0E0B0E0809331
:1003D000650090936600A0936700B0936800209337
:1003E0007D0030937E0040937F00509380001092F8
:1003F0007C0060936C0078C082E09ED59927AA2784
:10040000BB27082F192FFF24EE2483E095D59927C9
:10041000AA27BB27BA2FA92F982F8827E80EF91EE5
:100420000A1F1B1F84E088D5E80EF11C011D111D59
:10043000E0928900F0928A0000938B0010938C0068
:1004400085E07AD59927AA27BB27082F192FFF24E3
:10045000EE2486E071D59927AA27BB27BA2FA92FAA
:10046000982F8827E80EF91E0A1F1B1F87E064D506
:10047000E80EF11C011D111DE0926500F09266006E
:10048000009367001093680088E056D580936C0055
:1004900090917C0018166CF490937000ECD48093CB
:1004A0007C0080916C00ACD4B92FA82F972F862F99
:1004B00013C0923049F48091650090916600A0913C
:1004C0006700B091680008C08091890090918A000F
:1004D000A0918B00B0918C0080937D0090937E0062
:1004E000A0937F00B093800080917C00A6D2809181
:1004F0007D0090917E00A0917F00B0918000682FD8
:10050000792F8A2F9B2F71D380916C00181614F4C9
:100510001AD40DC080917D0090917E00A0917F0043
:10052000B0918000682F792F8A2F9B2F8ED37894DB
:10053000A8D480916A00882361F480918E0088237A
:1005400041F480917800882321F480916B00882306
:1005500089F0889580916A008823D9F780918E0070
:100560008823B9F780917800882399F780916B00F0
:10057000882379F7A895889584D4992781309105A7
:1005800019F0029761F1D0C080916C0018163CF40C
:100590008F5F80936C00833374F181E02AC0809177
:1005A000880020917D0030917E0040917F00509125
:1005B0008000882349F0B52FA42F932F822F8851D4
:1005C0009C4FAF4FBF4F57C08091790090917A00F8
:1005D000AA27BB27280F391F4A1F5B1F74C08091B1
:1005E0006C001816A4F5815080936C0018161CF04E
:1005F00082E380936C0080916D00882321F58091C7
:100600006C0039D480937C0080916C00F9D3B92FB1
:10061000A82F972F862F80937D0090937E00A09324
:100620007F00B093800080917C0007D280917D0094
:1006300090917E00A0917F00B0918000682F792F6B
:100640008A2F9B2FD2D280916C007DD38BC080915A
:10065000880020917D0030917E0040917F00509174
:100660008000882331F1B52FA42F932F822F885E2D
:100670009340A040B04080937D0090937E00A09373
:100680007F00B093800028EE33E040E050E0682F18
:10069000792F8A2F9B2F4AD2B92FA82F972F862FD9
:1006A00080937D0090937E00A0937F00B0938000A4
:1006B00012C08091790090917A00AA27BB27281B4D
:1006C000390B4A0B5B0B20937D0030937E004093E7
:1006D0007F00509380008091790090917A00AA2742
:1006E000BB27E0907D00F0907E0000917F0010918C
:1006F0008000282F392F4A2F5B2F912F802F7F2D9D
:100700006E2D14D2B92FA82F972F862F80937D009E
:1007100090937E00A0937F00B0938000682F792F84
:100720008A2F9B2F62D211C080916C001816D4F4CE
:1007300080916E0090916F000097A1F001979093C7
:100740006F0080936E00892B69F480917D009091F9
:100750007E00A0917F00B0918000682F792F8A2FB2
:100760009B2F73D220918E00222309F43FC09091D9
:100770006C001916ECF080916D008823C9F421E01B
:1007800020936D00892F992787FD909590958195ED
:100790009F4F80936C00882311F420936C0080910C
:1007A0006C008150823308F48FC020936C008CC0A1
:1007B00080916D00882309F4BCCE10926D00809169
:1007C0007D0090917E00A0917F00B0918000282F45
:1007D000392F4A2F5B2F60917C0080916C0067D38A
:1007E00080916C00992787FD909513C080917800C7
:1007F000882309F496C02093880080916D00909121
:100800006C00882361F020936D00892F992787FD64
:100810009095909581959F4F80936C0000C119161B
:100820000CF456C080917C0020917D0030917E00B8
:1008300040917F0050918000823049F42093650000
:1008400030936600409367005093680008C020937F
:10085000890030938A0040938B0050938C008093E2
:100860007000892F992787FD9095909581959F4FCE
:1008700080936C008150823318F081E080936C008B
:1008800080916C00F8D280937C0080916C00B8D28B
:10089000B92FA82F972F862F80937D0090937E00ED
:1008A000A0937F00B093800080917C00C6D080919F
:1008B0007D0090917E00A0917F00B0918000682F14
:1008C000792F8A2F9B2F91D180916C003CD231CE11
:1008D000892F992787FD9095909581959F4F8093BB
:1008E0006C008091700080937C00823049F480918C
:1008F000650090916600A0916700B091680008C003
:100900008091890090918A00A0918B00B0918C0019
:1009100080937D0090937E00A0937F00B093800031
:100920006EC090916C001916D4F080916B008823F2
:10093000B1F080917C00823090F48091880091E049
:10094000892780938800882321F080917700806830
:1009500003C0809177008F7780937700EACD1916D6
:100960000CF4E7CD80916A00882309F4E2CD10925F
:10097000880080917C00882311F481E023C02091BD
:100980007D0030917E0040917F0050918000813049
:10099000E1F42093890030938A0040938B005093B8
:1009A0008C008091650090916600A0916700B091E5
:1009B000680080937D0090937E00A0937F00B093A9
:1009C000800082E080937C001AC020936500309301
:1009D0006600409367005093680080918900909171
:1009E0008A00A0918B00B0918C0080937D00909341
:1009F0007E00A0937F00B093800010927C008091D5
:100A00007C001BD080917D0090917E00A0917F00A2
:100A1000B0918000682F792F8A2F9B2FE6D080918C
:100A20007D0090917E00A0917F00B0918000682FA2
:100A3000792F8A2F9B2F09D17CCDF894992781306B
:100A4000910519F0029749F148C0939868E975E05B
:100A50008FE0A7D188EE93E0A0E0B0E08093610042
:100A600090936200A0936300B093640080EE93E9DA
:100A7000A4E0B0E08093810090938200A093830073
:100A8000B093840089E190E090937A00809379009C
:100A90008AE080937700949A47C094986CEF7DE049
:100AA0008FE07FD184E694E1A0E0B0E08093610024
:100AB00090936200A0936300B093640082EA9FE386
:100AC000A0E0B0E08093810090938200A093830027
:100AD000B09384008AE590E01FC0949868E975E0BF
:100AE0008FE05FD188EE93E0A0E0B0E080936100FA
:100AF00090936200A0936300B093640080EE93E94A
:100B0000A4E0B0E08093810090938200A0938300E2
:100B1000B093840082E390E090937A008093790010
:100B20008CE080937700939A78940895AF92BF9267
:100B3000CF92DF92EF92FF920F931F93E62EF72E44
:100B4000082F192FA22EB32EC42ED52E609161002E
:100B5000709162008091630090916400E616F70640
:100B600008071907C8F16091810070918200809197
:100B70008300909184006E157F058007910760F1D6
:100B8000912F802F7F2D6E2DEBD1262F372F482FC1
:100B9000592F6115710581059105D1F0BD2DAC2D41
:100BA0009B2D8A2DB695A795979587952817390778
:100BB0004A075B0748F0A21AB30AC40AD50AEA0C2E
:100BC000FB1C0C1D1D1D04C0E21AF30A040B150BBF
:100BD000912F802F7F2D6E2D1F910F91FF90EF9001
:100BE000DF90CF90BF90AF900895262F372F482FDA
:100BF000592F203385E0380782E0480780E0580706
:100C000010F0C19801C0C19A20533242494F5F4F42
:100C100080917C00823049F4952F842F732F622FAE
:100C20002AE030E040E050E008C0952F842F732F79
:100C3000622F29E130E040E050E092D1F894732F28
:100C4000622F80E1AED078940895CF92DF92EF9238
:100C5000FF920F931F93CF93DF93E62EF72E082F6B
:100C6000192FF894C6E7D0E0CC2EDD2E912F802FDF
:100C70007F2D6E2D2AE030E040E050E071D1B92F99
:100C8000A82F972F862FFD2DEC2D80832197912F54
:100C9000802F7F2D6E2D2AE030E040E050E060D1C3
:100CA000E22EF32E042F152F0894C108D108F0E08E
:100CB000C137DF07DCF690916C00191624F08091A3
:100CC0007C008230B1F0191644F480916D008823C5
:100CD00021F4892FD0D0823061F080916C001816F9
:100CE00074F480916D00882351F080917C008230F3
:100CF00031F480917200882339F48FE003C0809131
:100D0000720080688093720080917100882319F4CA
:100D10008FE08093710080917500806880937500EA
:100D200080916C0018162CF080917600806880937A
:100D300076007894DF91CF911F910F91FF90EF9003
:100D4000DF90CF900895382FF8948FE08093710052
:100D500080937200809373002AE020937400832FA5
:100D6000622FF1D080937500832F622FECD0909387
:100D70007600832F45D0B92FA82F972F862F885E16
:100D80009340A040B04029F0809176008068809325
:100D9000760078948EEE92E090936F0080936E00D0
:100DA000089520B3207415BAC09896988D9A979894
:100DB00090E1891738F077FF02C0959A01C09598A5
:100DC000969A9698660F771F915099F7979A9598EB
:100DD0008D982111969A80918500882311F4C09AEC
:100DE00008958091850026E030E0281B310981E0DC
:100DF00090E002C0880F991F2A95E2F785BB0895FD
:100E0000CF92DF92EF92FF920F931F93CF93C82E52
:100E1000DD24C7FCD094CC0CDD1CCC0CDD1C8C2D4F
:100E2000895FCC2DC85F88D09927AA27BB27082FB8
:100E3000192FFF24EE248C2FCF5F7ED09927AA276D
:100E4000BB27BA2FA92F982F8827E80EF91E0A1F53
:100E50001B1F8C2F71D0E80EF11C011D111D912F4D
:100E6000802F7F2D6E2DCF911F910F91FF90EF90CE
:100E7000DF90CF900895880F880F8A5F5DD0992703
:100E8000089580916000992783709070880F991F52
:100E9000880F991F20B32370282B20936000E22F26
:100EA000FF27E45EFF4FC895802D99270895CF92C4
:100EB000DF92EF92FF920F931F93CF93E22EF32EC8
:100EC000042F152FC82EDD24C7FCD094CC0CDD1CBC
:100ED000CC0CDD1C8C2D8A5FCC2DC95F1DD0912FD1
:100EE000802FAA27BB272C2FCF5F682F822F14D0EB
:100EF000BB27A12F902F8F2D2C2FCF5F682F822FF4
:100F00000BD06E2D8C2F08D0CF911F910F91FF9099
:100F1000EF90DF90CF9008951F93CF93C82F162F97
:100F20000BD0811731F0E199FECFCEBB1DBBE29A09
:100F3000E19ACF911F910895E199FECF8EBBE09A7F
:100F40008DB39927089587FB082E062687FD819586
:100F500067FD61952CD00EF4919507FC819508955D
:100F6000A1E21A2EAA1BBB1BEA2FFB2F0DC0AA1F42
:100F7000BB1FEE1FFF1FA217B307E407F50720F002
:100F8000A21BB30BE40BF50B661F771F881F991F7D
:100F90001A9469F76095709580959095262F372F54
:100FA000482F592F6A2F7B2F8E2F9F2F0895991B23
:100FB00079E004C0991F961708F0961B881F7A9550
:060FC000C9F780950895B9
:00000001FF
